:050E0900323237430006
:100D650075A4CF75D40875F2F875A5F875A71F7524
:100D7500B0FF75A0FF7590FF7580FF75E10675E200
:020D850040220A
:0A0DF60075A14075F801E4F5A22292
:030E1200020DA925
:020E1500D322E6
:100CA300C207C208E4F5D9120D65120DF6120E152E
:100CB3009207300735120E127BFF7A0E790912085C
:100CC30000EF24FF92083008107D007C06E4FFFE4D
:100CD300120D1BE4FFFE120984E4FFFE0FBF0001A7
:0C0CE3000EBE27F8BF10F5E4F5C080FE3F
:090E000023213230304546550033
:0B0CEF0090005CEFF0FD90005BE0FF68
:050CFA00900079EDF00F
:100CFF00120D87EFC454F090007AF0900079E0FF66
:0B0D0F00120D8790007AE02FF0E0FF4B
:010D1A0022B6
:0B080000900067EBF0A3EAF0A3E9F022
:10080B0090007174FFF0A3740EF0A37400F09000CD
:10081B006E7401F0A37400F0A37408F090006A12D8
:10082B000C7200000000E47F50FEFDFC90006AE0BB
:10083B00F8A3E0F9A3E0FAA3E0FBC3120C50504A73
:10084B0090006AA3A3A3E0FF7BA0E4FD120B08902A
:10085B00006EE0FBA3E475F001120C3AA9F0FAEF7D
:10086B00120C2890006AE0FCA3E0FDA3E0FEA3E0DD
:10087B00FFE4FAF9F8EF2401FFEA3EFEE93DFDE85B
:10088B003CFC90006A120C66809C900071E0FBA30C
:10089B00E0FAA3E0F9120BE2FF900008E06F706240
:1008AB00900001120BFBFF900009E06F7054900059
:1008BB0002120BFBFF90000AE06F704690000312D0
:1008CB000BFBFF90000BE06F7038900004120BFBDA
:1008DB00FF90000CE06F702A900005120BFBFF904D
:1008EB00000DE0B5071C900006120BFBFF90000EED
:1008FB00E0B5070E900007120BFBFF90000FE06FA7
:10090B0060037F0022900067E0FBA3E0FAA3E0F90D
:10091B00120BE2FF900019E06F702A900001120B8E
:10092B00FBFF90001AE0B5071C900002120BFBFFB7
:10093B0090001BE0B5070E900003120BFBFF90001D
:10094B001CE06F60037F0022900011E0900004F028
:10095B00900012E0FFA3E0900006CFF0A3EFF09021
:10096B000021E0900000F0900022E0FFA3E0900057
:08097B0002CFF0A3EFF07F01B1
:010983002251
:100DA90075B283E4F5A9538EF4758920758DF975AB
:0B0DB9008BFFD28E75C15D43C180220C
:100D1B008F828E83D3E5829DE5839C5019758F035B
:100D2B0075B7A575B7F1E4F0F58F2582F5827402DE
:060D3B003583F58380DE24
:010D4100228F
:0B0B0800900074EFF0A3EDF0A3EBF001
:100B1300C2052009FDD209C200D201D203D2047F4B
:100B230001C2C4C206D2C530C0FDE5C054F0248062
:100B3300606224C0601A24E06003020BC790007651
:100B4300E0F5C2A200E43342C2C2C5E4A3F080765A
:100B530030C136300606D2C5C206806A30010CC2E7
:100B630001D202900075E0F5C2805B300211C2022F
:100B7300900074E0F5C230034DD206D200804720C6
:100B83000044E4900077F0803D300404D2C5803601
:100B9300D2058032EFFD900077E0FB3395E0FAC396
:100BA300EB9D7480F86A98500CA3E5C2F09000772F
:100BB300E004F0D2C1900077E0B5070AC209C2C1D0
:100BC300D2C48002D20530050853C0BF43C040C21F
:0E0BD30009C2C0300903020B2A900078E0FF2F
:010BE10022F1
:100D420090005BEFF0900065E0FEA3E0FF120DDD86
:080D5200900065EEF0A3EFF044
:0A0D5A00EEFD900001E0FB120B0813
:010D6400226C
:100DC400900004E0FFA3E0C39F500D900001E024D5
:090DD40002F0900005E004F02299
:100DDD000FBF00010EC3900007E09F900006E09E3C
:090DED005006120DC4E4FEFF22C1
:08098400900058EEF0A3EFF023
:10098C00E490005BF0A3F0900061F0A3F0900065A0
:10099C00F0A3F0900002E0FFA3E0900065CFF0A37D
:1009AC00EFF0900000E0A3F0E490005CF090005BAE
:1009BC00F090000504F0E4900060F090005BE064BF
:1009CC003A6025900065E0FEA3E0FF120D5A9000FE
:1009DC005BEFF0900065E0FEA3E0FF120DDD9000F0
:1009EC0065EEF0A3EFF080D3900062E004F07006A7
:1009FC00900061E004F0900065E0FEA3E0FF120DB2
:100A0C005A120D42120CEF90005EEFF09000601243
:100A1C000D46120D42120CEF900063E4F0A3EFF0C0
:100A2C00900063A3E0FFFD900060E02DF0EF9000DC
:100A3C0063F0A3E4F0A3120D4A120D42120CEF90D6
:100A4C000063E0FEA3E04FFF900063EEF0FEA3EF27
:100A5C00F0AC068C08F509900060E02F120D4612E0
:100A6C000D42120CEF90005DEFF0900060E02FF063
:100A7C00EF706990005AF090005EE0FF90005AE031
:100A8C00C39F5058120D47120D42120CEF90005F8D
:100A9C00EFF0A3E02FF0A3E0B4010AA3E0B4DA0571
:100AAC00E490005BF0D3900059E09509900058E079
:100ABC009508501F758F0175B7A575B7F190005F3C
:100ACC00E0850982850883F0E4F58F0509E5097056
:100ADC0002050890005AE004F0020A83120D471236
:100AEC000D42120CEF90005FEFF0A3E02F700C9012
:0B0AFC00005DE0640160030209C222FB
:010B070022CB
:040E0E0002000022BC
:03000000020600F5
:03000300021A03DB
:03000B00021A06D0
:03001300021A09C5
:03001B00021A0CBA
:03002300021A0FAF
:03002B00021A12A4
:03003300021A1599
:03003B00021A188E
:03004300021A1B83
:03004B00021A1E78
:03005300021A216D
:03005B00021A2462
:03006300021A2757
:03006B00021A2A4C
:03007300021A2D41
:10060000E4F5D9E5EF7480F5FF7402F5EF787FE447
:10061000F6D8FD9000007F007E04E4F0A3DFFCDE4E
:07062000FA758121020CA311
:100BE200BB010689828A83E0225002E722BBFE0211
:090BF200E32289828A83E4932244
:100BFB00BB010CE58229F582E5833AF583E02250AF
:100C0B0006E92582F8E622BBFE06E92582F8E222F8
:0D0C1B00E58229F582E5833AF583E4932212
:100C2800BB010689828A83F0225002F722BBFE01AB
:020C3800F322A5
:100C3A00A3F8E0C5F025F0F0E5821582700215836D
:060C4A00E0C838F0E822CA
:100C5000EB9FF5F0EA9E42F0E99D42F0EC6480C81B
:060C600064809845F022BB
:0C0C6600ECF0A3EDF0A3EEF0A3EFF02201
:100C7200A8828583F0D083D082120C89120C89124B
:100C82000C89120C89E473E493A3C583C5F0C58370
:100C9200C8C582C8F0A3C583C5F0C583C8C582C8CC
:010CA200222F
:100D8700EF7E0024D0B40A00401624F9B40A0040CC
:100D97000CB41000400A24E0B41000400374FFFEB6
:020DA700FF2229
:00000001FF
